:100000000AC018951895189518951895189518956B
:100010001895189518958FED8DBFC0ECE0EC4E2E1D
:10002000DD275D2EEEE7F0E0A0E6B0E088278D93B7
:100030003197E9F792D266248FEF81BB8EE187BBBF
:10004000C09AC59AC69AC79AC29AC19AE4E6F0E0E5
:1000500080E4CBD258E0C895802DC1D231965A9514
:10006000D1F704C00C12120C20202020E4E8F0E0AC
:1000700080E5BBD258E0C895802DB1D231965A9513
:10008000D1F704C020201F1F1F1F20204CD28CE05E
:10009000ACD2E6E9F7E03FD2E2E0F0E055D243D25D
:1000A000E6EAF7E038D23DD2ECEAF7E034D2E3E01A
:1000B000F0E04AD238D2EAE0F0E0AAE656D3E4E132
:1000C000F0E0ABE652D3EFE0F0E0A6E64ED3EFE08F
:1000D000F0E0A0E14AD3043608F00EC024D2ECEBE5
:1000E000F7E019D21ED2E6E9F7E015D2C498C3981A
:1000F00085B7806385BF8895C298FBD1FAD180E02F
:100100008093600080E08093610081E080936800CC
:1001100000916800083010F009F01CC0A1E60C91B5
:1001200042E02DD34C93E5D10091610040916000F5
:10013000040FA1E60C93B09B04C081E080936000A3
:1001400003C080E080936000A8E68C918F5F8C9361
:1001500008F4DECFC29A84E690E073D2C198C9D188
:10016000C8D180E08093600080E08093620081E0ED
:100170008093680000916800083010F009F01CC0FE
:10018000A2E60C9142E0FBD24C93B3D10091620005
:1001900040916000040FA2E60C93B09B04C081E084
:1001A0008093600003C080E080936000A8E68C919B
:1001B0008F5F8C9308F4DECFC19A84E690E041D241
:1001C000A3E68C918F5F8C93009163000E3108F051
:1001D00001C04FC080E08093630040916A000091AD
:1001E0006100041708F405C0809167008F7B80933D
:1001F000670000916A0042E0041BACE60C9340915A
:100200006C0000916100041710F009F005C08091A6
:10021000670080648093670040916B0000916200EA
:10022000041708F405C0809167008F7D80936700F4
:1002300000916B0042E0041BADE60C9340916D0011
:1002400000916200041710F009F005C0809167006A
:10025000806280936700A7E68C9186FBA8E38C916F
:1002600084F98C93A7E68C9185FBA8E38C9183F9A4
:100270008C938FE711E066D1EAECF7E04CD1009166
:1002800061000A3008F003C0EEECF7E044D1A8EAC0
:10029000B0E0E1E6F0E009D236D180E0A0D1E0EDB7
:1002A000F7E039D18FE71AE04DD1E4EDF7E033D133
:1002B000A8E38C9184FBA8EAB0E0D6D18D9388277F
:1002C0008C9321D18FEB11E03DD1EAEDF7E023D102
:1002D000009162000A3008F003C0EEECF7E01BD199
:1002E000A8EAB0E0E2E6F0E0E0D10DD180E077D11D
:1002F000E0EDF7E010D18FEB1AE024D1EEEDF7E05E
:100300000AD1A8E38C9183FBA8EAB0E0ADD18D932C
:1003100088278C93F8D0BE98A7E69C9194FF04C0E0
:10032000B69B0EC09F7E9C93B6990AC089E19F93AD
:10033000992787D19F91B69903C090619C9304D06F
:1003400084EF91E07ED1C3CEEFE0F0E0A6E60DD2DF
:1003500080916600815080936600EFE0F0E0A6E6B1
:100360007BE7F2D1809167008F7780936700DBD0C5
:10037000E4EEF7E0D0D0D5D0E8EEF7E0CCD0BD98F1
:10038000A7E69C9193FF04C0B59B0EC0977F9C93FA
:10039000B5990AC089E19F93992753D19F91B59947
:1003A00003C098609C9329D0BF98A7E69C9192FFC8
:1003B00004C0B79B0EC09B7F9C93B7990AC089E18C
:1003C0009F9399273ED19F91B79903C094609C93C6
:1003D00052D0EAE0F0E0AAE67BE7B6D1E4E1F0E053
:1003E000ABE67BE7B1D1A7E68C9187FB0EF001C0AD
:1003F000089584E690E025D1C2CF80E080936A0022
:1004000092D0B69906C0809167008068809367009B
:100410000895B59907C084E690E013D1AAE68C91BF
:100420008F5F8C938FE711E08DD0E6EFF7E073D00C
:1004300000916A000A3008F003C0EEECF7E06BD0E0
:10044000A8EAB0E0EAE6F0E030D15DD080E0C7D0C5
:1004500080916A008093690000916A00033610F071
:1004600009F001C004C080E080936A005CD084E69B
:1004700090E0E7D0C6CF80E080936B0054D0B6996F
:1004800006C0809167008068809367000895B799DF
:1004900007C084E690E0D5D0ABE68C918F5F8C935B
:1004A0008FE711E04FD0EAEFF7E035D000916B0015
:1004B0000A3008F003C0EEECF7E02DD0A8EAB0E077
:1004C000EBE6F0E0F2D01FD080E089D080916B00A5
:1004D0008093690000916B00033610F009F001C0B1
:1004E00004C080E080936B001ED084E690E0A9D029
:1004F000C6CF969AEF93FF93E6E0F0E096D0FF9197
:10050000EF9196980895A8EAB0E08D91882311F0B4
:1005100066D0FBCF0895A4D0802D11F060D0FBCF22
:10052000089580EC62C081E060D014D080E85DC0A6
:100530008FE7213039F08FEB223021F08FE8233024
:1005400009F08FEC810F51C088EE93E07AD031979B
:10055000D9F7089583E0992774C08AEF90E071D0AD
:100560008D9A8C9A8B9A8A9A899A889A909885E023
:1005700090E067D0919895989498939A929A919ACE
:10058000EF93FF93E0E6F0E050D0FF91EF91919868
:1005900055D0919AEF93FF93E0E6F0E046D0FF91BB
:1005A000EF9191984BD0919AEF93FF93E0E6F0E0B2
:1005B0003CD0FF91EF91919841D09298919AEF930E
:1005C000FF93E0E6F0E031D0FF91EF91919836D0C3
:1005D00088E20BD08EE009D086E007D00895909A8B
:1005E000829505D004D02AD008959098F9CF8595AA
:1005F00010F4929A01C09298859510F4939A01C0D4
:100600009398859510F4949A01C09498859510F468
:10061000959A01C09598919AEF93FF93E0E6F0E0E8
:1006200004D0FF91EF91919808953197F1F70895D3
:10063000689462F80895E89462F8089581E090E083
:1006400000C0EF93FF93EE27E82BE92B31F0E8EEA3
:10065000F3E03197F1F70197D1F7FF91EF9108950A
:10066000C89531960020089580E30EF4839508958F
:10067000000F111F221F331F08950095109520951C
:1006800030950F5F1F4F2F4F3F4F089501911081FD
:100690000EC001911191219130810BC00191108107
:1006A00017FF05C03FEF2FEF04C00081112722275D
:1006B000332737FF03C0E1DF8DE28D93CF93DF93C4
:1006C000CF92DF92EF92AA24BB24CC24DD24EE2427
:1006D00040E2CAE0DD2755E093E38881890F87FD7A
:1006E0009F7083FD907F891B89935A95A9F7C0DF7E
:1006F000AA1CBB1CCC1CDD1CEE1C4A9551F7E894CF
:10070000EFE0FF2782910ED0EB30E0F71EF0689407
:100710008A2D0CD088278D93EF90DF90CF90DF91BA
:10072000CF910895982F829501D0892F8F70805D89
:1007300026F0803309F4089568948D930895E19923
:10074000FECFEEBB3196089591E001C092E07B3779
:1007500051F47FB7F894F3DF8D918DBBE29AE19A63
:100760009A95C9F77FBF7727089591E001C092E07D
:10077000E6DFE09A8DB38D939A95D1F70895FF93B4
:100780005527F8E0469508F4500F57954795FA9588
:10079000D1F7FF9108955757572E4156522E344D99
:1007A000472E434F4D0044454D4F000047534D3AAF
:1007B00030343020383332313739000044454D4F22
:1007C0002045585049524544000054313A00200019
:1007D000432000004F7574313A0054323A004F758F
:1007E00074323A00536574003C54313E3C4F4B3EEA
:0E07F0003C54323E000054313D0054323D0076
:00000001FF
